:1000000000308A00712800001030840000080319B5
:10001000182801308D008C018C0B0C288D0B0B28BF
:100020004A308C008C0B122800000000800B09283D
:1000300000348316061283120612831605108312EB
:1000400005108316851083128510643090000420FB
:1000500000348316861283128612831606138312C7
:1000600006176430900004208316061283120616C9
:1000700083160510831205148316851083128514C8
:100080000034831686128312861683160613831293
:100090000617643090000420831606128312061699
:1000A0008316051083120514831685108312851498
:1000B000A4288316861283128612831606138312CF
:1000C000061364309000042083160612831206166D
:1000D0008316051083120514831685108312851468
:1000E000B12884011F3083058E0101308F008316F3
:1000F0008612831286128316061383120617643043
:1001000090000420831686148312861889280130F3
:100110008E0083160614831206188F288E010F088E
:100120000E020319B4280E08FE3E0318B428023E3E
:10013000B62883160511831205151920292064306D
:1001400090000420192041288F01B428192029206B
:1001500064309000042083160511831205111920C4
:10016000592801308F00B428822863000A108A10B1
:080170000A1182079928A62854
:02400E00F93F78
:00000001FF
